:10000000830100308A004A28F60003088301AD000E
:10001000831203130C1F11280D289F1F112810286D
:10002000132812284328A00A6D30AC00AC08031D29
:100030001A281B281C28242883120313AC03AC089D
:10004000031D232824281C280000000000000000B5
:100050006D3083120313AC00AC08031D3028312827
:1000600032283A2883120313AC03AC08031D392845
:100070003A28322800000000000000008312031319
:100080001F08AB000C13031383122D088300F60E18
:10009000760E0900203084002D3053208301C62DB8
:0E00A00004068001840A040603190034502867
:100AE200732DAD258312031328080319A903A80344
:100AF200280A0319290A031D7F2D802D722D031345
:100B020083120800F401F5010310F30CF20C031C2C
:100B1200912D7008F40771080318710AF507031084
:100B2200F00DF10D7208730403190034852D0530A0
:100B320083120313A100A108031DA02DA12DA22D34
:100B4200AA2D83120313A103A108031DA92DAA2D07
:100B5200A22D0313831208006D3083120313AA001F
:100B6200AA08031DB52DB62DB72DBF2D8312031371
:100B7200AA03AA08031DBE2DBF2DB72D0000000039
:100B8200000000000313831208008316031386017A
:100B9200053083129F00313090008B1783160C179B
:100BA2000B178B130130831286001230A800A901A3
:100BB2007125023086001230A800A9017125043087
:100BC20086001230A800A901712508308600123073
:100BD200A800A9017125103086001230A800A901D1
:100BE2007125203086001230A800A90171254030FD
:0E0BF20086001230A800A9017125803086000F
:100C00001230A800A9017125403086001230A800DA
:100C1000A9017125203086001230A800A901712594
:100C2000103086001230A800A90171250830860016
:100C30001230A800A9017125043086001230A800E6
:100C4000A9017125023086001230A800A901712582
:100C5000013086000A30A800A901712586011230F2
:100C6000A800A90171258B17FE2F831203130F080B
:100C7000A2000E08A1007A302202133003192102CB
:100C8000031C432E442EFE2F8E018F018B13200850
:100C9000A300A0018B17F030F2000030F30023080E
:100CA000F000F10183257408F0007508F1000030B0
:100CB000F11BFF30F200F3007008A4007108A500DA
:100CC0007208A6007308A70000302702031D722EC9
:100CD00000302602031D722E01302502031D722EE4
:100CE000F43024020318752E762E772E86010030FC
:100CF000831203132702031D872E00302602031DD3
:100D0000872E01302502031D872EF4302402031C98
:100D10009C2E8A2E00302702031D982E00302602BA
:100D2000031D982E05302502031D982EDC30240269
:100D300003189C2E9B2E9E2E9D2EA02E01308600E9
:100D40000030831203132702031DB02E0030260249
:100D5000031DB02E05302502031DB02EDC30240209
:100D6000031CC52EB32E00302702031DC12E0030F8
:100D70002602031DC12E09302502031DC12EC430D9
:100D800024020318C52EC42EC72EC62EC92E03302A
:100D900086000030831203132702031DD92E003072
:100DA0002602031DD92E09302502031DD92EC43079
:100DB0002402031CEE2EDC2E00302702031DEA2E37
:100DC00000302602031DEA2E0D302502031DEA2EF7
:100DD000AC3024020318EE2EED2EF02EEF2EF22E64
:100DE000073086000030831203132702031D022FF1
:100DF00000302602031D022F0D302502031D022F95
:100E0000AC302402031C172F052F00302702031DCE
:100E1000132F00302602031D132F11302502031D4E
:100E2000132F943024020318172F162F192F182F61
:100E30001B2F0F3086000030831203132702031D7F
:100E40002B2F00302602031D2B2F11302502031DEE
:100E50002B2F94302402031C402F2E2F003027020A
:100E6000031D3C2F00302602031D3C2F15302502A8
:100E7000031D3C2F7C3024020318402F3F2F422FAC
:100E8000412F442F1F3086000030831203132702A6
:100E9000031D542F00302602031D542F1530250248
:100EA000031D542F7C302402031C692F572F003060
:100EB0002702031D652F00302602031D652F193000
:100EC0002502031D652F643024020318692F682F43
:100ED0006B2F6A2F6D2F3F30860000308312031373
:100EE0002702031D7D2F00302602031D7D2F1930A0
:100EF0002502031D7D2F64302402031C922F802FB6
:100F000000302702031D8E2F00302602031D8E2F76
:100F10001D302502031D8E2F4C3024020318922F02
:100F2000912F942F932F962F7F30860000308312BD
:100F300003132702031DA62F00302602031DA62F30
:100F40001D302502031DA62F4C302402031CBB2F8D
:100F5000A92F00302702031DB72F00302602031DE2
:100F6000B72F21302502031DB72F34302402031878
:100F7000BB2FBA2FBD2FBC2FBF2FFF3086000030F4
:100F8000831203132702031DCF2F00302602031DF7
:100F9000CF2F21302502031DCF2F34302402031C14
:100FA000E42FD22F00302702031DE02F003026024D
:100FB000031DE02F25302502031DE02F1C302402E5
:100FC0000318E42FE32FE62FE52FE82FF8308600F3
:100FD0000030831203132702031DF82F003026026E
:100FE000031DF82F25302502031DF82F1C30240285
:100FF000031CFB2FFC2FFE2FC0308600352E4A2805
:02400E00503F21
:00000001FF
